:10000000012F2843294F4B31484D41C0D0C0E00556
:100010001BE51BB40707751B00B2B3D200D0E0D0BC
:02002000D032DC
:10002300C0D0C0E0E599F51FC298011D75815551F7
:10003300BF712D51FE30B502B1AEB1D830B54720F6
:10004300050FE524B43C0AD2057169118F71801143
:100053008F3000E6C20020B3E1D190200204C2B287
:100063000169D2B2516F0521E521B43CCD75210060
:1000730005220524E522B523C1752200713B118FAA
:100083007152118F013D71A2B174013DC2ACC29C8A
:10009300C2B2C2B4D2997925E7B4240E3099FDC215
:1000A30099D2B2D2B4D29CD2AC22B4266EE51EB49D
:1000B300001C09E71975F003A4F5F03128F51CE5D8
:1000C300F0043128F51EE5F004043128F51DE51C84
:1000D300FFE51DFE20E704B1F901E2EF317FFD15D5
:1000E3001E051CE51EB4000709EDB4242E212519B5
:1000F300EDB424070909751E002125B4231DE50D60
:10010300B40006750D05750E08150DE50DB4000256
:100113002119051E151CA80EE6050E3099FDC2997E
:10012300F59909019B0483220002000201000307E1
:10013300000A09061307001A090A2307002A0912ED
:100143003307003A09224307004A090A5307005AB2
:1001530009126307006A092200FF010012801212CC
:10016300802412803612804812805A12806C1280CA
:100173007E1280901280A21280B439800483220DF3
:100183000A303A496E74657276616C206D696E3A15
:10019300200D0A313A527963686C6F73742073656A
:1001A300723A200D0A323A4D7963616C6C2020203B
:1001B30020203A20200D0A333A426561636F6E3185
:1001C3002020746F3A20200D0A343A426561636F30
:1001D3006E31207669613A20200D0A353A42656115
:0101E30063B8
:1001E4006F6E31207669613A20200D0A363A4265F5
:1001F40061636F6E322020746F3A20200D0A373A03
:10020400426561636F6E32207669613A20200D0A7F
:10021400383A426561636F6E32207669613A202014
:100224000D0A393A426561636F6E20746578743AD9
:100234000D0A4D696E692D57582053746174696FA6
:100244006E202A2041544D454C2070726F636573B3
:100254006F722070726F6772616D6D656420627970
:1002640020284329204F4B31484D4175082D200249
:100274000D75092D750A2D750B2D750C2D2275081C
:1002840020750920750B2E750C30E51030030575AB
:10029400082DF404C3135003750C3575F06484B44D
:1002A40001042430F508740AC5F084B4000241B88E
:1002B4002430F509E5F02430F50A22758921751BEF
:1002C40000752100752200751E00750D007524004F
:1002D400C205C20451ECD1FFB1E551E3C2B32275AA
:1002E400B80275A892D28C22758DFD758BFDD28EC5
:1002F400759850C299C298D29C22750F00915F756F
:100304001E00912B9430540F75F00AA4F523051C9C
:10031400912BB4240975F00AE52384F52322943043
:10032400540FFDE5232DF523227E007FFFB1F9ED67
:10033400B42C0122F15C22900341719722C0002663
:100344000426022606260803F026100DC024900376
:1003540058719722C000260A2602260C260E03F0A6
:1003640026100DC02490036F719722C00026042626
:10037400022606260803F0261B0DC024900386716E
:100384009722C000260A2602260C260E03F0261BFE
:100394000DC0247925E493F709A3B424F822E51FBA
:0103A400B4A4
:1003A500000122E51EB4005BE51F751F0075F00016
:1003B500B43002813F75F001B43102813F75F0031D
:1003C500B43202813F75F005B43302813F75F00701
:1003D500B43402813F75F009B43502813F75F00BE5
:1003E500B43602813F75F00DB43702813F75F00FC9
:1003F500B43802813F75F010B43902813FB40D0263
:10040500C20422E51FB40D047424C2049135151EDF
:10041500051C751F00EDB4240CE51D30E104917B2E
:10042500B110751E0022E51CFFE51DFEB1F9ED2298
:10043500FDE51CFFE51DFED10022E5F0F50F752554
:100445000D75260A752726F52875290D752A0A754D
:100455002B3D752C3E752D24118FE50F75F003A4EA
:10046500F5F03128F51CE5F0043128F51EE5F0041A
:10047500043128F51D22915F912BB4240CE51CC392
:100485009407F51C7424913522151E151E151EE5BD
:100495001CC39407F51C74409135051CD51EF7E562
:1004A5001D75F06020E20F75F0E020E30975F0613D
:1004B50020E40375F061E5F09135915F151E151E79
:1004C500912BB4240122B42D29051C912BB4310D97
:1004D500051C912BB42404743181E2240AC39430A1
:1004E500540FC333C0E0915F151C912BD0E04D91A3
:1004F5003522C333FDE51CC39407F51CED9135E5A5
:100505001C2407F51C051CD51EB622750F0E915F20
:10051500912B750F0DB4240A915F151C912BD2E018
:10052500A12F915F151C912BC2E09135750F089194
:100535005F912B750F07B4240A915F151C912BD27F
:10054500E0A150915F151C912BC2E09135750F0606
:10055500915F912B750F03B4240A915F151C912BA4
:01056500D2C3
:10056600E0A171915F151C912BC2E0913522200408
:1005760009D2049005817197118F220D0A26112642
:1005860000261226012613260326142605261526DE
:1005960007261626092617260B2618260D2619269F
:1005A6000F261A26100D0A247402FFE4FEB1F9ED97
:1005B600C394305407F9B1CDF58D7407B5010443E2
:1005C60087802253877F22048322A0D0E8F4F8FA9A
:1005D600FDFD30010122D201C297D297C20122D27B
:1005E60001B1F0D109D116C20122D297D296C29496
:1005F600C29522D201D153C20122D201D109D138EA
:10060600C20122C294C2977406D176C294D29722AE
:10061600C294C2977401D1767400D176C294D297EF
:10062600D16C22C294C2977405D176D184C294D279
:100636009722C294C29774028EF0A2F092E3D1760A
:10064600EFD176EDD176C294D297D16C22C294C204
:100656009774038EF0A2F092E3D176EFD176D1842F
:10066600FDC294D297227999D12930E002D9F92294
:100676007808C294339295D294D8F7C29522780816
:10068600D294C294A29633D8F722D1FFF106400243
:10069600C1BBF11DF118D1FFF1064002C1BBF11D2E
:1006A600F122E5196002C1BBD202E511B4FF03D203
:1006B6000322C20322C20222D1C07FB7DFFE227FFD
:1006C60028DFFE227F1CDFFE227F03DFFE227E085C
:1006D600C2AFC29300D293D1CFA29392E003D1CA04
:1006E600D2AFDEEC227E08A2E0C2AFC2939293D1D3
:1006F600C5D293D2AF03DEEF22C293D1BED29322EC
:100706007E3C309306D1CFDEF9C322D1CFDEFCA2E8
:1007160093227444D1EB2274CCD1EB2274BED1EB7C
:010726007959
:10072700107809751A00D1D4F7F13809D8F8A71A43
:1007370022C0E0C0F0C0E075F008651A13E51A5052
:1007470002641813F51AD0E003C0E0D5F0ECD0E04E
:10075700D0F0D0E0229007767E007F00E16AFDD1DD
:10076700000FA3E493B426F67D2C7FFFD10022313E
:1007770024379E9660AEB040614F4B3057582420C7
:100787002020829898404040E0414C4C2420202073
:100797002020244040404040612420202020202069
:1007A700202024202020202020242020202020203A
:1007B7002020829898404040E0414C4C2420202043
:1007C700202024202020202020242020202020201A
:1007D700202024202020202020242020202020200A
:0307E700202026A9
:00000001FF
